:10000000CBC01EC2E3C0E2C0E1C0E0C0DFC0DEC0C2
:10001000DDC0DCC0DBC0DAC0D9C0D8C0D7C0D6C014
:10002000D5C0D4C0D3C022032800530029004E00FD
:10003000450053002F004100740061007200690008
:100040005F00550053004200180372006100700009
:1000500068006E00650074002E006E00650074007C
:10006000040309040902220001010080320904008E
:100070000001030000000921010100012200000726
:1000800005810308000A0A033600300032003200FE
:1000900005010905A1010901A10009300931150077
:1000A00026FF00750895028102C00509190129087B
:1000B00015002501750195088102C012010101009A
:1000C0000000088117970A040101020301050109D4
:1000D00002A1010901A10005091901290215002544
:1000E00001950275018102950175068103050109DB
:1000F0003009311581257F750895028106C0C0122F
:10010000010101000000088117990A04010102039E
:100110000105010905A1010901A1000930093115F5
:100120000026FF00750895028102C0050919012902
:10013000041500250175019504810275019504815E
:1001400003C0120101010000000881179B0A04018D
:100150000102030105010905A1010901A1000930FE
:100160000931150026FF00750895028102C0950629
:100170007501810305091901290215002501750181
:1001800095028102C012010101000000088117964A
:100190000A0401010203010011241FBECFE5D4E0CF
:1001A000DEBFCDBF10E0A0E6B0E0ECECF1E102C0B4
:1001B00005900D92A23BB107D9F711E0A2EBB0E098
:1001C00001C01D92A231B107E1F759C319CFCF93F6
:1001D000DC01C62F693008F0C8E02BE49091CA001A
:1001E00090FD23EC8091620087FF04C09F5F909395
:1001F000CA0003C08FEF809362002093FB00ECEFF6
:10020000F0E02C2F21502F3F19F08D918193FACFE0
:100210006C2F8CEF90E0C6D2CC5FC0936200CF9180
:1002200008951F93CF9390910B01992309F48CC0EB
:10023000935097FD87C0E2EBF0E0E091FA00EF5FAA
:1002400040E0C0E8809108018D3209F077C0983015
:1002500009F074C08081807609F06DC025EF30E030
:100260004093F5008181882321F44093F60042E019
:1002700057C0853021F4828180930C0151C08630B3
:10028000D9F5C0EC8381813039F440910D01209182
:10029000F8003091F90044C0823021F442E224E6B3
:1002A00030E03EC08330C9F48281882321F444E0E9
:1002B00020E630E035C0813021F448E128E430E028
:1002C0002FC0823021F442E226E230E029C08330A0
:1002D00039F54AE026E830E023C0813221F449E0D4
:1002E00026E730E01DC08232D9F44091F70020911A
:1002F00010013091110114C0883021F441E02FE049
:1003000031E00EC0893021F4828180930F0108C052
:100310008A3011F441E004C08B3011F44093CA00DC
:1003200030930A01209309018781882339F486815B
:10033000841720F402C0CF0139D2482FC093C800DF
:100340004093640010920B01909164009F3F09F468
:100350004FC08091630087FF4BC0692F993008F030
:1003600068E0961B909364001BE48091C80080FDB8
:1003700013EC8F5F8093C800ADEEB0E0E09109010F
:10038000F0910A01962F915086FF13C09F3FB9F05C
:1003900084919D012F5F3F4FAF014F5F5F4F9150A1
:1003A000ED57F04011F48091F7008C93D901FA01D8
:1003B000EDCF9F3F21F081918D939150FACFF09333
:1003C0000A01E09309017727C62F693040F48DEECA
:1003D00090E0E8D19C2F9C5FC83030F402C01EE151
:1003E00092E08FEF809364001093EC009093630091
:1003F00080B3857019F01092C90011C08091C900B6
:10040000882369F494E680B3857049F49150D9F754
:1004100081E08093C90090930C0190930701CF91E4
:100420001F91089582EB90E0809306010B968093D4
:10043000FA0085B7836085BF8BB780648BBF089552
:100440000F930FB70F93809BFECF809B06C0809BBE
:1004500004C0809B02C0000000C01F933F932F93F5
:1004600031E014E000B3102710FD32E0102F3A9570
:10047000C9F700FDE7C000B3102717952FE72795B0
:10048000DF9310B3012707952795CF93C0910601FD
:1004900000B31027179527953BE0D0E04F9310B39A
:1004A0000127079527954FEF000055C0809BFECF91
:1004B000809B06C0809B04C0809B02C0000000C0DF
:1004C000DF9100C0CDCF10B3157079F1407C2C6F57
:1004D00013C000B3057049F141782C6F15C0057049
:1004E00021F1102F2C6F00B319C000B30570E9F093
:1004F0004E7F2C6F18C038F300B30570B1F0102791
:1005000017952795243028F310B3012707952795D1
:10051000422749934FEF00B3243008F31027179573
:100520002795243010F310B31570E1F101270795DA
:1005300027952430F0F000B30570A1F1102717952E
:1005400027952430E0F010B30127079527953A95B9
:1005500041F12430D0F000B3057021F11027179538
:1005600027952430C0F010B3012707952795243034
:10057000C2CF10B31570B1F04C7F2C6FDCCF00B33D
:10058000057081F0487F2C6FDECF10B3157051F0ED
:10059000407F2C6FE0CF00B3057021F0407E2C6FC0
:1005A000E2CF3DC03C2FC09106013C1B00E433303C
:1005B0000ABFA8F108811981412F1F7720910701F7
:1005C0000D3289F1013E79F10936C1F00777033424
:1005D00031F510910E01112311F100910B01003042
:1005E000D1F53430DAF130930B011093080100910A
:1005F000FA00C093FA000093060130C0121779F494
:1006000047FD3AC0309163003F3F29F10FEF00935F
:100610006300CCEED0E025C0002700930E014F917F
:10062000CF91DF910FC01217B9F700930E010FEFB2
:1006300000936400009363004F91CF910AB706FDC9
:1006400035CFDF9100E40ABF2F913F911F910F91A9
:100650000FBF0F911895C0E6D0E002C0C1E6D0E010
:1006600032E05F9302B30A7F016002BB55E011B331
:10067000156011BB20E819C0309162003F3F59F36B
:100680000FEF00936200CBEFD0E0EBCF052710E037
:1006900002BB10C0052710E0089402BB13C0052759
:1006A00010E015C0052710E019C020FF052702BB88
:1006B000279517951C3F50F720FF0527279502BB6C
:1006C00017951C3F38F720FF05272795179502BB84
:1006D0001C3F28F720FF0527279517951C3F02BBD5
:1006E00008F700C0499120FF052702BB2795179501
:1006F0001C3F80F520FF0527279502BB17951C3F5F
:1007000068F520FF05272795179502BB1C3F58F574
:1007100020FF0527279517951C3F02BB38F5242F8E
:100720003A9519F60A7F5F9102BB32E03A95F1F7EC
:1007300010910C01C256D04011F0109307010160D6
:1007400011B31A7F02BB0A7F4F91CF9111BB02BB3D
:10075000DF9178CF052710E002BBCACF052710E054
:10076000089402BBCDCF052710E0CFCF052710E0BE
:10077000D3CFA82FB92F8FEF9FEF41E050EA615000
:1007800070F02D9138E0722F7827969587952695F1
:1007900070FF02C0842795273A95A9F7F0CF80957E
:1007A00090950895E6DF8D939D930895FC012DECBF
:1007B00030E030930A0120930901808199278076E7
:1007C0009070809719F58181813081F4E091CB00A0
:1007D000F091CC000088F189E02DC9010995E091E4
:1007E000CB00F091CC00808199270895823049F4A4
:1007F00083ED90E090930A018093090181E090E0FD
:1008000008958A3019F483818093D30080E090E0CA
:100810000895EF92FF920F931F93CF93DF93AC0154
:10082000415050408FEF4F3F580711F180E3E82EC1
:1008300085E7F82E012D112D23E130E0C701019746
:10084000F1F72150304037FFF9CFA0E3B5E7C0E022
:10085000D0E021E330E0CD010197F1F721503040A5
:1008600037FFF9CF415050408FEF4F3F580721F7E6
:10087000DF91CF911F910F91FF90EF900895CFE5F9
:10088000D4E0DEBFCDBFC0E001E01C2FB89A87B333
:10089000897F87BB88B3866088BBC09880E395E773
:1008A0000197F1F786B3992786709070002E02C0E9
:1008B000959587950A94E2F78230910591F08330FF
:1008C00091051CF4019749F002C0039791F05FD4A1
:1008D0009093CC008093CB0021C081E090E099DF21
:1008E000FCCFF9D39093CC008093CB0081E090E0D3
:1008F00014C051D1FC019093CC008093CB000284B2
:10090000F385E02D0995E8D1882329F068D39093E9
:10091000CC008093CB0082E090E07BDFE091CB00C5
:10092000F091CC0084819581909311018093100106
:1009300082818093F70080859185009731F09093B4
:10094000F9008093F800868107C085E891E09093D4
:10095000F9008093F8002AD480930D0114BA8FEF28
:1009600085BB98EF92BB95E091BB90E09150F1F779
:100970008150D9F781BB85E083BF8FE085BD84ECD2
:1009800083BDE091CB00F091CC000284F385E02D93
:10099000099548DD7894A89544DC002349F0E0915E
:1009A000CB00F091CC000484F585E02D099500E0A2
:1009B00008B600FE0CC091E098BF8091D300882358
:1009C00031F0153010F0155002C0182FC92F08B69D
:1009D00007FE18C080E888BFCC23A1F4E091CB00CB
:1009E000F091CC000484F585E02D0995E091CB00D1
:1009F000F091CC000684F785E02D0995882359F203
:100A0000C1E002C0CC2339F2809162008F3F19F619
:100A1000C0E0E091CB00F091CC000088F189E02D9E
:100A20008DEC90E00995E091CB00F091CC006081D5
:100A30008DEC90E0CCDBAFCF90E0AC9A80E38A9570
:100A4000F1F7AC9828E130E040E050E067E070E07A
:100A5000822F8A95F1F7AD98990F9B9B9160822F19
:100A60008A95F1F7AD9A6150704077FFF1CF90937E
:100A7000D40028E130E040E050E067E070E0822FF1
:100A80008A95F1F7AD9896959B9B9068822F8A95F1
:100A9000F1F7AD9A6150704077FFF1CF9093D50098
:100AA00008951F931FB7F894A49AA59AA398AB9A98
:100AB000AD9AAC98C1DF1FBF1F9108958091770058
:100AC00090917800892B39F010927800109277007D
:100AD00021E030E00BC042E050E066ED70E084EDD4
:100AE00090E067D3282F332727FD3095C90108955B
:100AF000CF93DC01892B09F444C08091D400C091CC
:100B0000D50060E870E0FB01482F552740FF02C088
:100B1000EFEFF0E041FF02C0E0E0F0E042FF02C092
:100B20006FEF70E043FF02C060E070E0EC93FD0106
:100B300061839A01220F232F221F330B3195CA01A3
:100B400080749070A5E095958795AA95E1F7282B7C
:100B5000CA018072907073E0959587957A95E1F758
:100B6000282B4071507055954795242B8C2F992731
:100B70008F70907034E0880F991F3A95E1F7282B19
:100B800022838091D4009091D5009093D7008093D8
:100B9000D600CF91089580E990E090936A00809309
:100BA000690085E690E00895FC01AC9A80E38A959F
:100BB000F1F7AC9828E130E040E050E097E0822F78
:100BC0008A95F1F7AD98822F8A95F1F7AD9A9150F9
:100BD00097FFF5CF28E130E040E050E097E0822F2A
:100BE0008A95F1F7AD988081880F80839B9902C028
:100BF00081608083822F8A95F1F7AD9A915097FF9B
:100C0000EECF0895AF92BF92CF92DF92EF92FF9214
:100C10000F931F93CF93DF93CDB7DEB721970FB616
:100C2000F894DEBF0FBECDBF46E0C42ED12C33E01A
:100C3000A32EB12CA822B922CE010196B5DF89815D
:100C400099278073907024E0959587952A95E1F710
:100C50008A159B0529F4B092DD00A092DC002BC020
:100C600088EB9BE00197F1F724E030E040E050E0B2
:100C700080E3E82EF12C012D112D6EE170E0AC9A8D
:100C8000822F8A95F1F7AD98AD9A822F8A95F1F768
:100C9000AC988E2D8A95F1F76150704077FFEFCFB9
:100CA00080E89BEB0197F1F70894C108D108C114C3
:100CB000D10409F0C1CF21960FB6F894DEBF0FBE64
:100CC000CDBFDF91CF911F910F91FF90EF90DF90FB
:100CD000CF90BF90AF900895CF93DF93CDB7DEB79D
:100CE00021970FB6F894DEBF0FBECDBFCE0101969F
:100CF0005BDF898199278F7090708130910511F0A9
:100D000080E090E021960FB6F894DEBF0FBECDBF15
:100D1000DF91CF9108950F931F93CF93DF93CDB7BA
:100D2000DEB721970FB6F894DEBF0FBECDBF10E03F
:100D3000012FCE01019638DF8981282F3327C90181
:100D40008F709070019761F54091DE005091DF0047
:100D50004115510551F5C90166E0969587956A954B
:100D6000E1F78130910591F0823091051CF4892BD7
:100D700049F00DC08230910521F0039741F4CA017A
:100D800005C040DF8091DC009091DD003BDFCE01AB
:100D900001960ADF898199278F709070019729F059
:100DA0001092DF001092DE0059C081E090E0909335
:100DB000DF008093DE0089818093E20080E797E185
:100DC0000197F1F780E08A95F1F740E250E060E0AA
:100DD00070E027E030E0842F8A95F1F7AD98110F8D
:100DE0009B9B11600000AD9A2150304037FFF3CF3C
:100DF00040E250E060E070E027E030E0842F8A9528
:100E0000F1F7AD98000F9B9B01600000AD9A215057
:100E1000304037FFF3CF202F2F77412F4F7707FD3B
:100E2000219517FD4195332727FD30958091DA00F4
:100E30009091DB00820F931F9093DB008093DA0088
:100E4000242F332727FD30958091D8009091D90029
:100E5000820F931F9093D9008093D80021960FB6EC
:100E6000F894DEBF0FBECDBFDF91CF911F910F91E0
:100E70000895A49AA59AA398AB9AAD9AAC984BDF23
:100E80008091E200992776E0969587957A95E1F72B
:100E90008130910569F0823091051CF4892B31F085
:100EA00008958230910531F0039729F480E090E0B5
:100EB000A9DE0895A7DE089540918B0050918C0023
:100EC0004115510529F010928C0010928B001CC026
:100ED0009091E2008091E3009817B1F42091DA003C
:100EE0003091DB008091E4009091E50028173907EC
:100EF00059F42091D8003091D9008091E60090916A
:100F0000E7002817390719F081E090E00895CA0139
:100F10000895FC01892B09F461C08091E000909153
:100F2000E100892B41F01082118212821092E100BF
:100F30001092E00008958091E2009927A6E096952E
:100F40008795AA95E1F780838091DA009091DB0084
:100F50002FEF8138920714F421E807C080389105FB
:100F600014F02FE702C02091DA008091D800909110
:100F7000D9003FEF8138930714F441E807C0803867
:100F8000910514F04FE702C04091D80021834283BD
:100F9000332727FD30953093E5002093E400552753
:100FA00047FD50955093E7004093E6008091E200A2
:100FB0008093E3008091DA009091DB00821B930B19
:100FC0009093DB008093DA008091D8009091D90053
:100FD000841B950B9093D9008093D80008958DECD5
:100FE00090E090937E0080937D008BEB90E0909357
:100FF00082008093810089E790E00895A49AA59AE1
:10100000A398AB9AAD9AAC98089590E0AC9A80E31F
:101010008A95F1F7AC9828E130E040E050E067E0D5
:1010200070E0822F8A95F1F7AD98990F9B9B9160A4
:10103000822F8A95F1F7AD9A6150704077FFF1CF1A
:101040009093E80008958091E8009091E900891B51
:10105000992787FD90950895FC01892BB9F120E827
:1010600030E0B9018091E800482F552740FF02C0C9
:101070006FEF70E041FF02C060E070E042FF02C02D
:101080002FEF30E043FF02C020E030E06083218397
:101090009A01220F232F221F330B3195CA0180742E
:1010A000907065E0959587956A95E1F7282BCA01C0
:1010B0008072907033E0959587953A95E1F7282BEB
:1010C0004071507055954795242B22838091E800FC
:1010D0008093E900089581E191E0909392008093DC
:1010E00091008FEF90E090939600809395008DE8AB
:1010F00090E0089584B3807F84BB85B38F6085BB07
:1011000087B38F7C87BB88B3806388BB089593B314
:101110009F7086B38073982B9093EB00089520E026
:1011200030E09091EB008091EA00981711F021E0F7
:1011300030E0C9010895FC01892B21F140E850E01D
:10114000BA018091EB008095282F332720FF02C041
:101150006FEF70E021FF02C060E070E022FF02C08C
:101160004FEF50E023FF02C040E050E06083418336
:10117000128224FF02C080E8828325FF03C082819F
:10118000806482838091EB008093EA00089584E577
:1011900091E09093A4008093A30082E491E0909367
:1011A000A8008093A7008FE990E0089582E190E085
:1011B0000895FB01DC0104C08D910190801921F498
:0C11C00041505040C8F7881B990B08955F
:1011CC005AD2FFFFFF03002B00000000000000516B
:1011DC00051C055E057805010003003200000012B5
:1011EC0000000039078B065C0789070100030031FA
:1011FC0000000012000000FE07050823082C08035D
:10120C000031000000120000007A0887088F089B4C
:02121C000800C8
:00000001FF
